:02000000D32803
:0A0006002A08AF000030B0000F30F0
:10001000AF070318B00A30088A002F0882000F3497
:10002000FB34CF343F34D03406340F34FB34CD347A
:100030008D34D03405340F34FB34CB34A534D03474
:100040000634A508031D2528080018300000FF3ECF
:10005000031D262800000000A50B25280800851098
:100060002508A2000310A20D2508A700A80103106F
:10007000A70DA80DA70A0319A80A00302802031D1E
:10008000432822082702031C6E280830A6002608F1
:10009000003C03186C282308A9002208AA000320AA
:1000A000AB002603AC000130AD00AE012C08FF39D7
:1000B0008A110A12031961280310AD0DAE0DFF3E1F
:1000C00057282D082B0503196728051568280511E1
:1000D00005120516A6034728A20A3428851408002D
:1000E000083083128B000930831696008C010F3084
:1000F00081003730950031308F003030831290000E
:100100007A3092009F0183169F0117308312990065
:100110009A012130831699001430831298001F3001
:100120008500093083168500831218108512851406
:1001300005160130A0000B1001300B05A4002008AB
:10014000240403199C280B100518B1280630A100BF
:100150002108083C031CC8282108A5002F20A10A5B
:10016000A828851DBE280330A1002108053C031CDA
:10017000C8282108A5002F20A10AB528A10121081F
:10018000023C031CC8282108A5002F20A10ABF2873
:1001900085160530A500212085121930A5002120E3
:1001A0000B10A0019C2801308312A0000030A30096
:0601B0008A110A127028FA
:02400E00D430AC
:00000001FF
